:020000040000FA
:060000008DEF06F0120076
:060800008DEF06F012006E
:06082A0001004E0D00006C
:080830000002000014000000AA
:08083800D9CFE6FFE1CFD9FFA3
:10084000020EE126DE6ADD6ADECF00F0DDCF01F0C8
:10085000FD0EDBCF02F0FE0EDBCF03F001500318DC
:10086000E8AE02D0033404D00250005C03500158BB
:100870000AE2010EE66E9BEC06F0E552DF2A010E5D
:1008800001E3DB2AE1D7020EE15C02E2E16AE55214
:10089000E16EE552E7CFD9FF1200D9CFE6FFE1CFF5
:1008A000D9FF040EE126DE6ADE6ADE6ADD6ADD5209
:1008B000DD52FB0EDBCF00F0FC0EDBCF01F0FD0EB6
:1008C000DBCF02F0FE0EDBCF03F0D9CFE9FFDACFAA
:1008D000EAFF030EEB500318E8AE02D0033408D051
:1008E0000050EE5C0150EE580250EE580350EE58A6
:1008F0000FE20C0EE66E6DEC06F0E552D9CFE9FF83
:10090000DACFEAFFEE2A000EEE22EE22EE22D1D757
:10091000040EE15C02E2E16AE552E16EE552E7CFE6
:10092000D9FF12000F0EC16E936A300E926E0F0E39
:10093000946E1200D9CFE6FFE1CFD9FF020EE12677
:100940008250020B01E0010E080DF3CF02F082503D
:10095000010B040DF3CF01F08050200B01E0010EDC
:10096000E824006E8050100B01E0010E00240124E9
:100970000224DE6EDD6ADECF00F0DDCF01F000C0C4
:10098000F3FF01C0F4FF020EE15C03E200D0E16A74
:10099000E552E16EE552E7CFD9FF120080920A0ED0
:1009A000E66EE66A49DFE552E55280840A0EE66E9D
:1009B000E66A42DFE552E55280940A0EE66EE66A88
:1009C0003BDFE552E552120080820A0EE66EE66ACF
:1009D00033DFE552E55280840A0EE66EE66A2CDFCC
:1009E000E552E55280940A0EE66EE66A25DFE5528E
:1009F000E5521200380E816ED1DF050EE66EE66A12
:100A0000E66AE66A4ADFE552E552E552E552010E32
:100A1000816EC4DF050EE66EE66AE66AE66A3DDFD1
:100A2000E552E552E552E5520D0E816EB7DF050E37
:100A3000E66EE66AE66AE66A30DFE552E552E552BE
:100A4000E552060E816EAADF050EE66EE66AE66ADC
:100A5000E66A23DFE552E552E552E5521200010E47
:100A6000816E9CDF050EE66EE66AE66AE66A15DFD1
:100A7000E552E552E552E5521200D9CFE6FFE1CF4B
:100A8000D9FF020E816E8ADF0A0EE66EE66AE66A1A
:100A9000E66A03DFE552E552E552E552FD0EDBCF93
:100AA000E6FFFE0EDB50280DF350E552E724E76E1B
:100AB000FE0EE7CFDBFFFD0EDB6AFE0EDB50F36EB2
:100AC000FD0EDBCFF4FFF350F45C0CE2140E816EEC
:100AD00065DF010EE66EE66AAFDEE552E552FD0E19
:100AE000DB2AEBD7E552E7CFD9FF1200D9CFE6FFDB
:100AF000E1CFD9FFFE0EDB50816E66DF0A0EE66E97
:100B0000E66A9ADEE552E552E552E7CFD9FF1200D8
:100B1000D9CFE6FFE1CFD9FFFD0EDBCFE9FFFE0E17
:100B2000DBCFEAFFEF500EE0FD0EDBCFE9FFDB2A63
:100B3000FE0EDBCFEAFF01E3DB2AEF50E66ED6DFE5
:100B4000E552EAD7E552E7CFD9FF1200EBDE52DFDC
:100B500086DFE66AE66A91DFE552E55202011E6B26
:100B60001F6B080E1FAF02D0D89003D01E5D000E81
:100B70001F590FE2000E1E25E96E020E1F21EA6EBC
:100B8000EF50E66EB3DFE55202011E2B000E1F236D
:100B9000E8D7E66A010EE66E70DFE552E552080E10
:100BA00002011E6F1F6B100E1FAF02D0D89003D032
:100BB0001E5D000E1F590FE2000E1E25E96E020E8B
:100BC0001F21EA6EEF50E66E91DFE55202011E2B07
:100BD000000E1F23E8D700C210F21E6B1F6B100E11
:100BE0001FAF02D0D89003D01E5D000E1F5919E22E
:100BF000010EEA6A1E25E96E1F51EA22000EE9265F
:100C0000020EEA22EF50E66E000E1E25E96E020E7D
:100C10001F21EA6EE552E750EF6E1E2B000E1F23D8
:100C2000DED7900EE66E010EE66EE66AE66A35DE07
:0C0C3000E552E552E552E5528CD7120067
:040C3C002A0EF66E18
:100C4000080EF76E000EF86E02010900F550196FDC
:100C50000900F5501A6F03E1196701D03DD0090072
:100C6000F550146F0900F550156F0900F550166F17
:100C700009000900F550E96E0900F550EA6E090017
:100C800009000900F550176F0900F550186F0900A9
:100C90000900F6CF1BF2F7CF1CF2F8CF1DF214C2F9
:100CA000F6FF15C2F7FF16C2F8FF0201175302E163
:100CB000185307E00900F550EE6E1707F8E2180721
:100CC000F9D71BC2F6FF1CC2F7FF1DC2F8FF0201D5
:0A0CD0001907000E1A5BBFD71200CF
:060CDA00FF0EE350066E60
:100CE000480E01D04C0EE76EE72EFED7E76AE72EDE
:0A0CF000FED7062EF7D70000120011
:060CFA00000EF36E00EE97
:100D000000F0080E01D81200EA6002D0EE6AFCD7AB
:0A0D1000F350E9601200EE6AFCD710
:060D1A0012EE40F022EE93
:100D200040F0F86A059C1EEC06F0A6EC06F0A6EC76
:060D300005F0FBD71200E4
:0A0D3600FF0EE350E84E120000002B
:0C0D400000D000D000D0E82EFAD712003E
:020D4C00120093
:020D4E00534907
:100D50005354454D4120424F4C5420563220000000
:020D6000000091
:00000001FF
